:02000000040AF0
:080008009F0C0200110A0A0C12
:100010002900F90C27000000E7020B0AE902090A8F
:100020000008080C0600080C2600020C2800010C31
:100030002600070907090709070907090709030C2B
:100040002600070907090709110C26000709E8021D
:10005000170A020C2800200C2600070907090709C7
:10006000070907090709210C2600070907090709DD
:10007000220C26000709E8022B0A020C2800100CAB
:100080002600070907090709070907090709300CAE
:100090002600070907090709110C26000709E802CD
:1000A0003F0A020C2800020C26000709070907096D
:1000B000070907090709120C26000709070907099C
:0C00C000220C26000709E802530A150A6A
:021FFE00EA0FE8
:00000001FF
